:020000040800F2
:10000000280A0020B10100084721000881170008D4
:1000100045210008290300089B2A00080000000071
:10002000000000000000000000000000292300087C
:100030002B030008000000004921000823260008C7
:10004000CB010008CB010008CB010008CB01000860
:10005000CB010008CB010008CB010008CB01000850
:10006000CB010008CB010008CB010008CB01000840
:10007000CB010008CB010008CB010008CB01000830
:10008000CB010008CB010008CB01000800000000F4
:10009000000000000000000000000000CB0100088C
:1000A000CB010008CB010008CB010008CB01000800
:1000B000CB010008CB010008CB010008CB010008F0
:1000C000CB010008CB010008CB010008CB010008E0
:1000D000CB010008CB010008CB01000800000000A4
:1000E000CB010008CB010008CB0100080000000094
:1000F000000000000000000000000000CB0100082C
:1001000000000000CB010008CB010008CB01000873
:1001100000000000000000000000000000000000DF
:10012000CB010008CB010008CB010008CB0100087F
:10013000CB010008000000000000000000000000EB
:10014000000000000000000000000000CB010008DB
:10015000CB010008CB010008CB010008CB0100084F
:10016000CB010008CB0100080000000000000000E7
:10017000000000000000000000000000000000007F
:1001800000000000CB01000800000000000000009B
:10019000CB010008CB010008DFF810D000F0B2F866
:1001A00000480047152D0008AFF30080280A002002
:1001B0000648804706480047FEE7FEE7FEE7FEE701
:1001C000FEE7FEE7FEE7FEE7FEE7FEE7B9260008EA
:1001D000990100082DE9F05F0546002092469B46F4
:1001E00088460646814640241BE02846414647464D
:1001F000224600F076F853465A46C01A914110D371
:1002000011461846224600F05DF82D1A67EB0108EA
:100210004F4622460120002100F054F817EB000958
:100220004E41201EA4F10104DFDC484631462A4637
:100230004346BDE8F09F40EA01039B0703D009E075
:1002400008C9121F08C0042AFAD203E011F8013BC2
:1002500000F8013B521EF9D27047D2B201E000F81B
:10026000012B491EFBD270470022F6E710B513465A
:100270000A4604461946FFF7F0FF204610BD421E0D
:1002800012F8013F002BFBD111F8013B02F8013BB2
:10029000002BF9D1704710B5002200E0521C835C9E
:1002A0008C5CA34201D1002BF8D1D8B2E1B2401A44
:1002B00010BD034611F8012B00F8012B002AF9D1DB
:1002C00018467047202A04DB203A00FA02F1002089
:1002D00070479140C2F1200320FA03F31943904084
:1002E0007047202A04DB203A21FA02F000217047EF
:1002F00021FA02F3D040C2F120029140084319468E
:1003000070470000064C074D06E0E06840F001032E
:1003100094E8070098471034AC42F6D3FFF740FF4B
:100320001C6A00083C6A0008FEE7704772B6FEE7E8
:10033000002229B101291AD002291BD04FF44072A2
:100340000E490B6823F440730B600B6813430B607A
:100350000A6822F0F8020A600A68022303EBC00070
:1003600002430A60086840F48030086070474FF428
:100370008072E5E74FF40072E2E70000103C0240B3
:100380001348016889050FD5016821F400710160E7
:10039000016841F400610160016821F400610160BD
:1003A000016841F400710160016849050FD50168D9
:1003B00021F480610160016841F4805101600168AD
:1003C00021F480510160016841F48061016070474F
:1003D000003C024038B50220009001240A4800F099
:1003E00031F9C0088440C4F58050009000F0D2F983
:1003F0000121009800F092F800F0C0F908B1022045
:1004000038BD012038BD000000C0000810B586B01E
:100410000B4800F017F904460020009002940948A8
:1004200000F010F9001B401C03900220049005A965
:10043000684600F057F9002800D0012006B010BD32
:1004400000C00008FFFF070800B587B00021029038
:100450000120039002200091049005A9684600F055
:1004600041F9002800D0012007B000BD10B50848B0
:1004700000F0E8F807490988C008C14040F6FF725B
:10048000C240914201D1012010BD002010BD0000EA
:1004900000C00008163C024010B500F07BF902498C
:1004A000F320086010BD00000C3C02402DE9F04133
:1004B00016468846054600240D4F11E058F82410D2
:1004C000286800F03BF82868016858F82400814249
:1004D00002D00220BDE8F0812868001D2860641C5D
:1004E000B44202D22868B842E8D90020F2E70000FE
:1004F000FBFF070808490A6822F440720A600A688C
:1005000042F004020A600A684FF4803343EA002094
:1005100002430A6070470000103C024010B50446D8
:100520004CF2503000F05AF8002803D102490A88F2
:1005300022430A8010BD0000163C0240074A13689F
:1005400023F440731360136843F40073136013685B
:1005500043F001031360016070470000103C02404B
:100560001C490868C2061C4805D5C26942F0100241
:10057000C26110220A600A68920605D5C26942F07B
:100580000802C26120220A600A68520605D5C269C3
:1005900042F00402C26140220A600A68120605D5D0
:1005A000C26942F00202C26180220A600A68D20572
:1005B00006D5C26942F00102C2614FF480720A603E
:1005C0000A68920705D5C26942F02002C261022082
:1005D000086070470C3C02400801002070B51149CA
:1005E00004460020C86100F0E5F906460E4D09E01A
:1005F000601C07D024B100F0DDF9801BA04201D9B6
:10060000032070BD2868C003F2D42868C00701D059
:1006100001202860286810F4F970F2D0FFF7A0FFDD
:10062000012070BD080100200C3C024008B50020EC
:100630008DF80000684601F06FFF0028FAD09DF8A1
:10064000000008BD01460020A1F100634FF4804284
:10065000934204D314480844904201D201207047C9
:1006600012480844904201D20220704710480844C2
:10067000904201D2032070470E480844B0F5803FF5
:1006800001D2042070470C480A184FF4003082420F
:1006900001D205207047094A1144814201D2062047
:1006A000704707207047000000C0FFF70080FFF789
:1006B0000040FFF70000FFF70000FEF70000FCF726
:1006C00070B5044600F076F90546601C02D0044877
:1006D0000078044400F06EF9401BA042FAD370BDCC
:1006E000000000202DE9F047044622480F46017E15
:1006F00001290AD00121804601764CF25039484642
:10070000FFF76CFF020003D02FE00220BDE8F08766
:100710004FF0FF3038602068174D012801D0A668DF
:100720001CE0207C6168FFF7E5FE4846FFF756FFB6
:100730000246286820F00400286014E0217C30463E
:10074000FFF7F6FD4846FFF749FF0200286820F052
:10075000FA00286001D03E6005E0761CD4E9021062
:100760000844B042EAD8FFF70BFE002188F81810C1
:100770001046CBE708010020103C024004480178F5
:1007800041F0020101704CF25030FFF727BF00002A
:10079000143C0240074900200A68002A09DA054A89
:1007A000054B0C3A1360054B13600968002900DA09
:1007B00001207047103C024023016745AB89EFCD13
:1007C0002DE9F84FDFF8B8A10022012403254FF0EE
:1007D0000F090AF1040BAAF1040E00BF0B6804FA1A
:1007E00002F63340B34273D10F7907F00307012FAC
:1007F00001D0022F16D187684FEA420805FA08FC9B
:1008000027EA0C07D1F80CC00CFA08FC4CEA070CDC
:10081000C0F808C04768B7430E79C6F30016964083
:100820003E4346600E79F643B6070DD0C7685600C2
:1008300005FA06FC27EA0C07D1F808C00CFA06FCFA
:100840004CEA070CC0F80CC00E7906F00306022E25
:1008500010D1D60800EB8608D8F8206057074FEA79
:10086000D76C09FA0CF7BE430F6907FA0CF7374348
:10087000C8F8207006684FEA420C05FA0CF7BE4330
:100880000F7907F0030707FA0CF7374307604E6844
:1008900016F4403F6DD03B4E376847F480473760D1
:1008A000366822F0030706F480460096364E07EBC2
:1008B000060CDCF8086897073F0F09FA07F826EAE4
:1008C0000806DFF8C880404503D14FF000081EE05D
:1008D0004FE0DFF8BC80404502D14FF0010816E040
:1008E000DFF8B080404502D14FF002080FE0DFF89A
:1008F000A880404502D14FF0030808E0DFF89C8053
:10090000404502D14FF0040801E04FF0070808FA13
:1009100007F848EA0608CCF80888DAF80060574675
:10092000D1F804C09E435FEACC2C00D51E433E6044
:10093000DBF800605F46D1F804C09E435FEA8C2C70
:1009400000D51E433E60DEF800607746D1F804C053
:100950009E435FEA8C3C00D51E433E60084F083F33
:100960003E68D1F804C09E435FEACC3C00D51E43EC
:100970003E60521C102AFFF431AFBDE8F88F000032
:10098000083C014044380240003001400000024071
:100990000004024000080240000C02400010024027
:1009A0000069084000D0012070470AB1816170479A
:1009B0000904FBE701488068704700000000002040
:1009C000024881680278114481607047000000206D
:1009D0000B4810B5016841F400710160016841F4F1
:1009E00080610160016841F480710160032000F0C2
:1009F00061F80F2000F006F800F024F8002010BD88
:100A0000003C024070B50D4D04464FF47A712878D1
:100A1000B1FBF0F00A490968B1FBF0F000F051FCBD
:100A200048B9102C07D200222146501E00F022F8AF
:100A300000206C6070BD012070BD0000000000202F
:100A40000C0000200A4808B5016841F480410160AB
:100A5000006800F4804000900548001F016841F0E4
:100A600080510160006800F08050009008BD0000D7
:100A700044380240F0B40E4B1B680C46C3F302230B
:100A8000C3F10705042D00D90425191D072901D23A
:100A9000002300E0DB1E012606FA05F1491E214075
:100AA00099409E40761E16403143F0BC02F0BCB81F
:100AB0000CED00E0064900F0070208684FF6FF035E
:100AC000184040EA0220034A1043086070470000C3
:100AD0000CED00E00000FA052DE9F0470E46050098
:100AE00065D0DFF81481D8F80000F7B200F00700F5
:100AF000B04207D288F80070D8F8000000F0070074
:100B0000B04254D128683D4C810712D5400703D527
:100B1000206840F4E05020602878000703D5206862
:100B200040F4604020602068A96820F0F00008438D
:100B300020602878C0072DD030496868083901281E
:100B400012D0022813D0032811D009688907002980
:100B50002DDA216821F0030101432160FFF72AFF0C
:100B6000814641F2883A0EE009688903EFE7096897
:100B70008901ECE7FFF71EFFA0EB0901514502D9FF
:100B80000320BDE8F0872068696800F00C00B0EB36
:100B9000810FEFD1D8F80010404601F00701B142B3
:100BA00007D90770006800F00700B04201D00120AB
:100BB000E7E72878400705D52068E96820F4E05089
:100BC000084320602878000706D52068296920F4AA
:100BD000604040EAC100206000F038F82168084A0F
:100BE000C1F30311515CC84006490860064800681B
:100BF000FFF708FF0020C4E7003C0240083802402D
:100C0000F06700080C00002004000020044805499B
:100C100000680968044AC1F38221515CC8407047EA
:100C20000C0000200838024000680008044805490C
:100C300000680968044AC1F34231515CC8407047FA
:100C40000C0000200838024000680008154810B564
:100C5000006810F00C02144813D01449042A0FD075
:100C6000082A0ED10F4C241F2268236802F03F028D
:100C70005B0207D52068C0F38810A0FB010106E0E5
:100C8000084610BD2168C1F38811A1FB00010023B3
:100C9000FFF7A0FA2168C1F30141491C4900B0FBEC
:100CA000F1F010BD083802400024F40040787D01C6
:100CB0002DE9F84F04006ED02078DFF84C93C00780
:100CC000A9F104054AD009F104000168C1F38101CA
:100CD000012908D00068C0F3810002280AD1D9F8A0
:100CE0000000400206D52868800337D560680028D8
:100CF000E1D033E06068B0F5803F10D0B0F5A02FB0
:100D0000286810D020F480302860286820F48020E3
:100D100028606068A8B1FFF74DFE06460DE0286820
:100D200040F48030F4E740F480202860F7E700BF0B
:100D3000FFF740FE801B642873D828688003F7D52E
:100D40000CE0FFF737FE064605E000BFFFF732FE76
:100D5000801B6428F0D828688003F7D42078DFF857
:100D6000AC8280074FF0000A3ED5A748001D0168FD
:100D700011F00C0F08D00068C0F3810002280BD1DD
:100D8000D9F80000400207D42868800716D5E0682B
:100D9000012800D112E033E1E068B8B10120C8F8C1
:100DA0000000FFF707FE064605E000BFFFF702FE62
:100DB000801B0228C0D828688007F7D528682169D9
:100DC00020F0F80040EAC10028600DE0C8F800A05B
:100DD000FFF7F0FD064604E0FFF7ECFD801B02285C
:100DE0001FD828688007F7D42078000722D5864FBF
:100DF00087486169703771B101210160FFF7DAFD41
:100E0000064604E0FFF7D6FD801B022809D83868A3
:100E10008007F7D50EE0C0F800A0FFF7CBFD06462F
:100E200005E082E0FFF7C6FD801B02287DD8386808
:100E30008007F7D42078400768D5DFF8CCB10027C9
:100E40000BF13C0BDBF80000C0000BD4DBF800100A
:100E500041F08051CBF80010DBF80000012700F0D2
:100E6000805000906B4E3068C00510D4306840F45C
:100E700080703060FFF79EFD009005E0FFF79AFD5F
:100E80000099401A022850D83068C005F6D55E4E49
:100E9000A0686C3601280FD00528306810D020F0EB
:100EA00001003060306820F004003060A068B8B104
:100EB000FFF780FD00900FE0306840F00100F4E79C
:100EC00040F004003060F7E7FFF774FD0099411A25
:100ED00041F28830814266D830688007F4D50EE050
:100EE000FFF768FD009007E0FFF764FD0099411AE5
:100EF00041F28830814256D830688007F4D42FB14F
:100F0000DBF8001021F08051CBF80010A069C8B3C5
:100F10003D49091D0968C1F3810102294AD002280F
:100F2000504607D0C8F8600000E03CE0FFF742FD03
:100F300004463BE04746C8F86000FFF73BFD064625
:100F400005E000BFFFF736FD801B02282BD828687C
:100F50008001F7D4D4E907010843A16A2E4A490861
:100F600002EB0141626A41EA8211084394F82C10B5
:100F700040EA0161C9F8001001203866FFF71AFD48
:100F8000044606E03EE000BFFFF714FD001B022808
:100F900009D828688001F7D534E000BFFFF70AFDC3
:100FA000001B022802D90320BDE8F88F28688001C1
:100FB000F4D427E00128F7D0D9F80000E26900F462
:100FC000800191421CD1226A00F03F01914217D169
:100FD00047F6C071626A0140B1EB821F10D1A26A6C
:100FE0004FF0FF3300F4403103EB5202B1EB024FFC
:100FF00006D194F82C1000F07060B0EB016F01D0B6
:101000000120D1E70020CFE704380240000047422A
:10101000800E4742007000400000FFFF70B50400E2
:1010200009D0606A002540B125616561A56294F828
:10103000510040B10CE0012070BD6068B0F5827FC6
:10104000F4D0E561F2E784F85050204600F044F80F
:10105000022084F851002068016821F040010160FD
:10106000A088218900F4827001F404410843A18919
:1010700001F400610843217C01F002010843217D55
:1010800001F001010843218B01F400710843217F25
:1010900001F03801084394F8201001F08001084362
:1010A000218D01F40051084321680860A0690421E2
:1010B00001EA104094F8241001F01001084321685F
:1010C00048602068C16921F40061C1616565012043
:1010D00084F85100002070BD10B586B0044614217C
:1010E0006846FFF7C1F814492068884221D11348A7
:1010F0000021026842F480420260006800F48040EF
:1011000005900E481038026842F002020260006842
:1011100000F0020005904FF4204000900220CDE93D
:101120000101032003900520049069460448FFF75D
:1011300047FB06B010BD00000038004040380240B8
:10114000000402402DE9F84F984616468A460446A8
:10115000FFF730FC814694F8510001281ED1BAF106
:10116000000F73D0002E71D094F85000012815D0D4
:10117000012784F85070032084F85100002565652C
:10118000C4F830A0A686E686A563A587E5876564D2
:101190002564A068B0F5004F03D00CE00220BDE844
:1011A000F88F2068016821F0400101602068016823
:1011B00041F48041016020680168490603D4016858
:1011C00041F040010160E068B0F5006F606803D055
:1011D00048B3012E27D047E008B1012E1FD1206B64
:1011E00021680088C86006E020688168890709D501
:1011F000216B0988C160206B801C2063E08E401E3B
:10120000E0860CE0FFF7D6FBA0EB0901414503D3D4
:10121000B8F1FF3F03D035E0B8F1000F32D0E08ED7
:101220000028E1D123E0206B21680078087306E0F4
:101230002068816889070AD5216B09780173206BC2
:10124000401C2063E08E401EE0860DE02BE0FFF79F
:10125000B1FBA0EB0901414503D3B8F1FF3F03D037
:1012600010E0B8F1000F0DD0E08E0028E0D14A4622
:101270004146204600F0C6FF08B120206065A06806
:1012800030B109E084F8517084F85050032086E7AB
:101290002068C1688068009084F8517004F8505F3D
:1012A00060680028F3D0012079E74FF0E02104289E
:1012B000086903D020F004000861704740F0040082
:1012C000FAE710B5401EB0F1807F01D3012010BDB8
:1012D0004FF0E02460610F21601701F0A5FC0020B1
:1012E000A06107202061002010BD10B590F83C20BF
:1012F000012A22D0012280F83C20CA688C6822F49E
:10130000407222434C6822F4806222430C6822F42B
:10131000006222430C6922F4805222434C6922F479
:1013200000522243C969002322F480420A43016823
:101330004A6480F83C30002010BD022010BD00003F
:1013400070B590F83C20012A2CD0012480F83C4054
:10135000022280F83D2003685A689D6822F07006DA
:101360000A6832435A60104B02689A420ED0B2F1BA
:10137000804F0BD00D4B9A4208D00D4B9A4205D0AE
:101380000C4B9A4202D00C4B9A4204D1496825F08A
:1013900080031943916080F83D40002180F83C10A3
:1013A000084670BD022070BD0000014000040040EE
:1013B00000080040000C00400040014010B586B01D
:1013C000044614216846FEF74FFF0E492068884204
:1013D00016D10D480021026842F001020260006847
:1013E00000F0010005904FF4806000900220CDE9EC
:1013F00001010120CDE9031069460448FFF7E0F937
:1014000006B010BD0000014030380240000002402C
:1014100070B5044690F83C0000260D4601280FD018
:10142000012084F83C006AB1042A1DD0082A2FD07C
:101430000C2A3FD00126002084F83C00304670BDC5
:10144000022070BD206801F09FF92068816941F099
:10145000080181612068816921F0040181612068AF
:1014600081692A69114311E0206801F0B5F920680B
:10147000816941F4006181612068816921F48061A2
:101480008161206881692A6941EA02218161D2E78C
:10149000206801F0CDF92068C16941F00801C161FF
:1014A0002068C16921F00401C1612068C1692A690D
:1014B000114311E0206801F0E7F92068C16941F4A7
:1014C0000061C1612068C16921F48061C161206847
:1014D000C1692A6941EA0221C161ACE710B5040083
:1014E00003D094F83D0010B107E0012010BD0020AA
:1014F00084F83C00204600F01FF8022084F83D00EC
:10150000211D206801F0E0F8012084F8460084F8ED
:101510003E0084F83F0084F8400084F8410084F8DD
:10152000420084F8430084F8440084F8450084F8BD
:101530003D00002010BD000008B500680649884243
:1015400008D10648016841F001010160006800F01F
:101550000100009008BD0000000001404438024036
:1015600010B50446022249B104290ED0082913D02F
:1015700094F84100012816D0012010BD94F83E00D7
:101580000128F9D184F83E200FE094F83F000128AB
:10159000F2D184F83F2008E094F840000128EBD114
:1015A00084F8402001E084F841200122206801F005
:1015B000DDF812492068884203D1426C42F40042AF
:1015C0004264206888420ED0B0F1804F0BD00C49A5
:1015D000884208D00B49884205D00B49884202D086
:1015E0000A49884204D1816801F00701062903D025
:1015F000016841F001010160002010BD00000140C0
:101600000004004000080040000C00400040014081
:1016100070B5040004D094F84100002510B106E034
:10162000012070BD84F84050204600F023F82420AB
:1016300084F841002068C16821F40051C16020464F
:1016400001F06CF92068016921F490410161206882
:10165000416921F02A0141612068C16841F40051CB
:10166000C1606564202084F8410084F8420065630D
:10167000002070BD10B586B0044614216846FEF700
:10168000F3FD14492068884221D1134800210268E3
:1016900042F020020260006800F0200005900E4831
:1016A0001438026842F001020260006800F0010094
:1016B00005904FF4C05000900220CDE901010320B5
:1016C00003900820049069460448FFF779F806B0B3
:1016D00010BD0000001401404438024000000240E8
:1016E0002DE9F843044690F84100984616460D4609
:1016F000202802D00220BDE8F88385B17EB1002009
:101700006064212084F84100FFF754F9A6848146E3
:10171000E684A0682027B0F5805F02D003E00120B6
:10172000E9E7206910B12E4600250EE000260CE006
:101730008021204601F078F9A8B9C6B116F8010B4E
:1017400021684860E08C401EE084E08C4B464FF0FE
:101750000002CDF800800028EAD14FF04001204679
:1017600001F062F940B184F841700320C3E735F815
:10177000020BC0F30800E3E784F841700020BAE7E9
:10178000FEE70000F0B500220D4B154614460A276F
:10179000B1FBF3F630368654B1FBF3F603FB1611BA
:1017A000B3FBF7F3521C861816F8016C302E00D1EB
:1017B00025B16D1C641C0A2CEAD3F0BD0022F9E7A8
:1017C00000CA9A3B00B587B014216846FEF74CFD6D
:1017D00009480021026842F001020260006800F03E
:1017E000010005900120CDE90001029069460348FF
:1017F000FEF7E6FF07B000BD3038024000000240AF
:101800002DE9F04104461D4616460F462A2000F0F9
:101810001BFA204600F008FA304600F005FA2B20AB
:1018200000F012FA384600F0FFF9284600F0FCF903
:10183000BDE8F0412C2000F007BA10B514460B4665
:101840000246FFF7DDFF2046BDE8104000F0ECB98E
:101850002DE9F04780461F46581E83B21646501E9B
:1018600082B20C464046DDF82090FFF7C9FF0AE03F
:10187000454604E0484600F0D7F96D1CADB2B542CC
:10188000F8D3641CA4B2BC42F2D3BDE8F0870000D8
:10189000F0B587B014216846FEF7E6FC18480168E9
:1018A00041F002010160016801F002010591016847
:1018B00041F00201016000684FF4805600F0020020
:1018C000059001240F4FCDE9006403256946039577
:1018D0003846FEF775FF012231463846FFF765F8B6
:1018E0002E02CDE90064084C694603952046FEF7B8
:1018F00067FF012231462046FFF757F807B0F0BDD9
:1019000030380240000402400000024070B5FFF78A
:10191000BFFF00224FF480716748FFF746F8674D1C
:101920004FF48054002221462846FFF73EF86420F9
:1019300001F0C0F9012221462846FFF736F864205D
:1019400001F0B8F9112000F07FF9782001F0B2F928
:10195000362000F079F9002000F08CF93A2000F0F0
:1019600073F9052000F086F9B22000F06DF90C2023
:1019700000F080F90C2000F07DF9002000F07AF9E9
:10198000332000F077F9332000F074F9B72000F02D
:101990005BF9352000F06EF9BB2000F055F91920F5
:1019A00000F068F9C02000F04FF92C2000F062F937
:1019B000C22000F049F9012000F05CF9C32000F0DA
:1019C00043F9122000F056F9C42000F03DF9202020
:1019D00000F050F9C62000F037F90F2000F04AF966
:1019E000D02000F031F9A42000F044F9A12000F04B
:1019F00041F9E02000F028F9D02000F03BF9042064
:101A000000F038F90D2000F035F9112000F032F91E
:101A1000132000F02FF92B2000F02CF93F2000F0CC
:101A200029F9542000F026F94C2000F023F9182061
:101A300000F020F90D2000F01DF90B2000F01AF93C
:101A40001F2000F017F9232000F014F9E12000F026
:101A5000FBF8D02000F00EF9042000F00BF90C2068
:101A600000F008F9112000F005F9132000F002F948
:101A70002C2000F0FFF83F2000F0FCF8442000F09C
:101A8000F9F8512000F0F6F82F2000F0F3F81F20AD
:101A900000F0F0F81F2000F0EDF8202000F0EAF848
:101AA000232000F0E7F8212000F0CEF8BDE87040D8
:101AB000292000F0C9B800000000024000040240E4
:101AC000411F5F2909D84FF4967110FB01F0642182
:101AD000B0FBF1F001490968C86370477800002045
:101AE0002DE9FF4F81B00446DDF83C9000904FEAAD
:101AF00059074FF00008780700D0012000EBD7000D
:101B000000FB09FB203AD0B20390029802994844A6
:101B1000401E83B2E019401E82B22046FFF770FEDD
:101B2000002553E0B9F10C0F2AD0B9F1100F2ED0D7
:101B3000B9F1180F2ED0B9F1200F49D127490398D8
:101B400001EB8010002610F805A0109800284FF037
:101B5000010000FA06F000EA0A0022D020B1204677
:101B6000049A0299FFF769FE641C0098A4B2201A37
:101B7000B84225D10298009C401C80B2029023E01C
:101B80000398174900EB400001EB8000DAE71549A4
:101B9000039803E00398144900EB400001EB0010A8
:101BA000D0E708B1049800E00E9800F03DF808F185
:101BB0000100C0B2B0FBF7F1804607FB118050B1C5
:101BC000761CF6B2082EC0D36D1CADB25D45A9D30C
:101BD00005B0BDE8F08F4FF00008F5E7084B0008AE
:101BE000D42E000848330008383900082DE9FE4F8C
:101BF0009946DDE90D6714468A460546DDF83080D2
:101C00000CE0CDF800804B4651462846CDE90167EF
:101C1000FFF766FF05EB560085B2641C2278002AA8
:101C2000EFD1BDE8FE8F000008B5010A8DF8001065
:101C30008DF801000123022269460248FFF782FA6B
:101C400008BD00002000002070B5094D06464FF485
:101C50000074002221462846FEF7A7FE304600F019
:101C600009F821462846BDE870400122FEF79DBED6
:101C70000000024001B501231A4669460148FFF7FA
:101C800061FA08BD20000020094808B5016841F04C
:101C900002010160016801F002010091016841F058
:101CA00001010160006800F00100009008BD000023
:101CB00030380240104810B50E4901604FF482716F
:101CC0004160002102228160C0E9031201224261C9
:101CD0005202C0E906210162416281620A21C162A9
:101CE000FFF79CF9002803D0BDE81040FEF71EBBAB
:101CF00010BD0000003800402000002010B592B058
:101D000000240F941C2108A81094FEF7ADFA20219E
:101D10006846FEF7A9FA20481E4901606321C0E920
:101D20000114FA21C0E9031444618461FFF7D6FB72
:101D300008B1FEF7FBFA0F940FA917481094FFF7AC
:101D4000FFFA08B1FEF7F2FA6020CDE908040A9420
:101D50000B940C940D94082208A90F480E94FFF7D9
:101D600057FB08B1FEF7E2FA00944FF40050CDE9BA
:101D70000440029401940394694607480794FFF7CE
:101D8000B4FA08B1FEF7D2FA0348FFF717FB12B016
:101D900010BD000000000140780000200C4810B584
:101DA0000A4901604FF4E1314160002181600C2259
:101DB000C160C0E904128161C161FFF729FC0028FC
:101DC00003D0BDE81040FEF7B1BA10BD00140140C9
:101DD000C0000020354800F0BBFB354800F0B8FBE0
:101DE000344800F0B5FB344800F0B2FB314800F055
:101DF000AFFB324800F0ACFB2C4800F0A9FB30A050
:101E000000F0A6FBFEF732FB2F4C002510B9012095
:101E1000206000E025602DA000F09AFB3BA000F0C0
:101E200097FB4AA000F094FB58A000F091FB2068BB
:101E300010B166A000F08CFB74A000F089FBFEF7E7
:101E4000F5FB312806D0322807D0332807D03428B4
:101E500014D016E000F06AFADDE77CA015E04FF040
:101E6000E02005614561856172B683494868A060DC
:101E70006060096881F308888047CCE72068012802
:101E800006D0206800280FD07CA000F061FBC2E7DC
:101E9000FEF7A0FA012803D00228BCD187A0F4E7FE
:101EA00091A000F055FBB5E797A0EEE7D0690008D8
:101EB000EC680008A0680008846900083869000818
:101EC0000D0A0D0A00000000100000200D0A3D3D23
:101ED0003D3D3D3D3D3D3D3D3D3D3D3D3D3D3D3D32
:101EE000204D61696E204D656E75203D3D3D3D3D47
:101EF0003D3D3D3D3D3D3D3D3D3D3D3D3D3D3D3D12
:101F00003D3D3D3D3D3D3D0D0A0A00002020446F12
:101F1000776E6C6F616420496D61676520546F2036
:101F20007468652053544D33324634787820496EB6
:101F30007465726E616C20466C617368202D2D2D66
:101F40002D2D2D2D20310D0A0A0000002020557066
:101F50006C6F616420496D6167652046726F6D200A
:101F60007468652053544D33324634787820496E76
:101F70007465726E616C20466C617368202D2D2D26
:101F80002D2D2D2D20320D0A0A000000202045782D
:101F9000656375746520546865204E6577205072BE
:101FA0006F6772616D202D2D2D2D2D2D2D2D2D2D39
:101FB0002D2D2D2D2D2D2D2D2D2D2D2D2D2D2D2D51
:101FC0002D2D2D2D20330D0A0A00000020204469FC
:101FD0007361626C6520746865207772697465202E
:101FE00070726F74656374696F6E202D2D2D2D2DA9
:101FF0002D2D2D2D2D2D2D2D2D2D2D2D2D2D2D2D11
:102000002D2D2D2D20340D0A0A0000003D3D3D3DB3
:102010003D3D3D3D3D3D3D3D3D3D3D3D3D3D3D3DF0
:102020003D3D3D3D3D3D3D3D3D3D3D3D3D3D3D3DE0
:102030003D3D3D3D3D3D3D3D3D3D3D3D3D3D3D3DD0
:102040003D3D3D3D3D3D0D0A0A0000005468697369
:102050002066756E6374696F6E206973206469739E
:1020600061626C65642120506C65617365205573F5
:102070006520310D0000000000C00008496E766147
:102080006C6964204E756D6265722021203D3D3E75
:1020900020546865206E756D6265722073686F7577
:1020A0006C642062652065697468657220312C203B
:1020B000322C2033206F7220340D00004572726F75
:1020C000723A20466C617368207772697465207576
:1020D0006E70726F74656374696F6E206661696C8F
:1020E00065642E2E2E0D0A00577269746520507299
:1020F0006F74656374696F6E2064697361626C6587
:10210000642E2E2E0D0A0000496E76616C696420E3
:102110004E756D6265722021203D3D3E20546865FC
:10212000206E756D6265722073686F756C642062D5
:10213000652065697468657220312C2032206F72C9
:1021400020330D00FEE7FEE7704770B50C460546EC
:1021500004E0284600F0E0F9012804D0641EF8D21B
:102160004FF0FF3070BD002070BD2DE9F84F88465C
:1021700000210646C8F80010924611466846FFF74F
:10218000E4FF4FF0FF39B0BB9DF80000182814D0D1
:1021900006DC012809D0022809D004282BD12EE022
:1021A000412816D0612826D113E0802401E04FF4A5
:1021B000806401253070671D15E051466846FFF7C1
:1021C000C4FFC0B99DF80000182814D1C8F80090C9
:1021D00015E00120BDE8F88F70195146FFF7B5FFF3
:1021E00048B96D1CADB2BD42F6D3B178707881F0BC
:1021F000FF01884201D04846ECE7C8F800400020C3
:10220000E8E70000F8B515460E460B460092044676
:102210000122022100F02CF8A0B9134813490068EC
:10222000B0FBF1F04FF47A71484300906068B0F56C
:10223000827F0DD13346002280212046009500F098
:1022400017F870B1606D40F0200060650320F8BDA4
:10225000009830B1401E009020688068C04300069E
:10226000F6D50020F8BD00000C00002000366E01FD
:102270002DE9F8431E46914688460446089DFEF720
:1022800099FB401B351AFEF795FB07462548006869
:10229000C0F3CB30684338E0701C37D0FEF78AFBC0
:1022A000C01BA84203D215B1009860B32CE020688F
:1022B000416821F0E00141606068B0F5827F0BD198
:1022C000A068B0F5004F02D0B0F5806F04D120684F
:1022D000016821F040010160A06AB0F5005F09D1FA
:1022E0002068016821F4005101602068016841F410
:1022F00000510160012084F85100002084F8500052
:102300000320BDE8F8830025401E00902068816806
:1023100038EA010004D000214945BDD10020F0E792
:102320000121F9E70C000020704700001FB520A232
:1023300007CA8DE80700214803900220FEF784F8C1
:102340001FA000F005F92D4800F0A8FB041E1FDDBA
:102350002B4800F0FDF82B4800F0FAF821466846BB
:10236000FFF710FA28A000F0F3F8684600F0F0F844
:1023700028A000F0EDF82AA000F0EAF82EA1022231
:1023800003A8FEF793F808B12EA00CE03C480AE041
:10239000601C05D0A01C05D0E41C07D039A002E0C9
:1023A00040A000E04FA000F0D3F81FBD54A0FAE712
:1023B0002020202020202020202000000080000855
:1023C00057616974696E6720666F72207468652052
:1023D00066696C6520746F2062652073656E742079
:1023E0002E2E2E202870726573732027612720748B
:1023F0006F2061626F7274290A0D000028010020AD
:102400004C680008280500200A0D2053697A653AB7
:10241000200000002042797465730D0A000000005E
:102420002D2D2D2D2D2D2D2D2D2D2D2D2D2D2D2DDC
:102430002D2D2D0A0000000041505020464C4147F0
:10244000000000000A0A0D2041505020466C6167D0
:1024500020536574204572726F72210A0D2D2D2D47
:102460002D2D2D2D2D2D2D2D2D2D2D2D2D2D2D2D9C
:102470002D2D2D2D2D2D2D2D2D2D2D2D2D0D0A00FC
:10248000086800080A0D4661696C656420746F2055
:1024900072656365697665207468652066696C6538
:1024A000210A0D000A0A0D54686520696D6167658F
:1024B0002073697A6520697320686967686572208E
:1024C0007468616E2074686520616C6C6F776564F8
:1024D000207370616365206D656D6F7279210A0DDF
:1024E000000000000A0A0D5665726966696361742E
:1024F000696F6E206661696C6564210A0D000000D9
:102500000D0A0A41626F72746564206279207573E6
:1025100065722E0A0D000000054909680A68D24359
:10252000920603D44968017001207047002070476B
:10253000C000002004494860044800680168C9439D
:102540000906FBD47047000000100140C0000020C5
:1025500000B5024603E000BFFFF7ECFF521C107805
:102560000028F9D100BD70B5002204781346302C44
:1025700004D14478782C0AD0582C08D06FF02F055D
:10258000845C74B36B2C2ED04B2C2CD030E0827832
:102590000AB30224025D5AB1A2F14105052D0AD900
:1025A000A2F16106052E06D91135092D07D913E0D0
:1025B00001200B6011E0A2F13006092E01D8303A5B
:1025C00004E0052D01D8373A00E0573A641C02EBCD
:1025D00003130B2CDED302E000200B2C00D30020D1
:1025E00070BD0B6002E01AB1980207E0012015E00F
:1025F0006D2C01D04D2C03D112B118050860F5E700
:10260000A4F13006092E08D803EB830305EB43033E
:10261000521C23440B2AB3D3E1E700200B2ADED25D
:1026200070BDFEF7CDB9000030B593B030216846DB
:10263000FDF71AFE14210CA8FDF716FE1C48002415
:10264000016841F080510160006800F080501190F5
:102650001848016841F4404101600068022500F417
:1026600040401190012003901020049000950695A1
:102670000820CDE907406420CDE9090504200B902E
:102680006846FEF715FB08B172B6FEE70F20CDE9EC
:102690000C054FF48050CDE90E4003210CA8109496
:1026A000FEF71AFA002801D072B6FEE713B030BD6B
:1026B00040380240007000400248016841F4700157
:1026C0000160704788ED00E0F0B50268204B214CB6
:1026D0009F03214D214E984207D0B84205D0A04219
:1026E00003D0A84201D0B04204D122F0700C4A6855
:1026F00042EA0C02984210D0B8420ED0A0420CD050
:10270000A8420AD0B04208D0154CA04205D0154CC2
:10271000A04202D0144CA04203D122F44074CA68F3
:1027200022434C6922F08002224302608A68C2621E
:102730000A688262984201D10969016301214161FD
:102740000169C90703D0016921F001010161F0BDF0
:10275000000001400004004000080040000C004060
:1027600000400140004401400048014010B501F024
:102770001F030121046A99408C430462016A9A4054
:102780001143016210BD000030B5036A026A22F0F5
:10279000010202624268846924F073050C682C43CC
:1027A00023F002058B682B430A4DA8420BD123F07E
:1027B0000805CB6822F440722B434D6923F00403D3
:1027C00015438A692A434260846149684163036210
:1027D00030BD00000000014030B5026A036A23F0FA
:1027E00010030362436884690D6824F4E64444EAF4
:1027F00005248D6822F0200242EA05120B4DA84202
:102800000ED1CD6822F0800242EA05124D6923F410
:10281000406343EA85038D6922F0400243EA850361
:102820004360846149688163026230BD00000140F9
:1028300030B5036A026A22F4807202624268C46997
:1028400023F4007324F073050C682C438D6843EA6D
:1028500005230C4DA8420ED1CD6823F4006343EA52
:1028600005234D6922F4405242EA05128D6923F492
:10287000806342EA05124260C4614968C163036231
:1028800030BD00000000014030B5046A026A22F445
:10289000805202624268C3690D6823F4E64343EA4A
:1028A00005238D6824F4005444EA0534064DA842FB
:1028B00004D14D6922F4804242EA85124260C3612C
:1028C00049680164046230BD0000014001680C31B8
:1028D00051E8002F22F4907241E80023002BF5D13B
:1028E0000168143151E8002F22F0010241E8002371
:1028F000002BF5D1016B012909D101680C3151E898
:10290000002F22F0100241E80023002BF5D12021F6
:1029100080F84210002101637047000070B5044642
:1029200000680169E26821F44051114301612169A5
:10293000A068E26908436169114308432168CA68D5
:1029400049F20C639A430243CA6020684169A26954
:1029500021F440711143416131492068884202D01D
:102960003049884202D1FEF761F901E0FEF74EF9E5
:10297000E2690023192164253226B2F5004F62680E
:1029800028D0A0FB0101930F9200FDF723FC014624
:10299000B0FBF5F06FF01802504301EB800006EB3E
:1029A0000010B0FBF5F000F0F002B1FBF5F002EB27
:1029B0000012B1FBF5F06FF01803584301EB8000F3
:1029C00006EB0010B0FBF5F000F00F00216810449A
:1029D000886070BDA0FB010192185B41FDF7FAFB16
:1029E0000146B0FBF5F00201B1FBF5F06FF0180302
:1029F000584301EB800006EBC000B0FBF5F000F09F
:102A0000F80002EB4002B1FBF5F0584301EB800007
:102A100006EBC000B0FBF5F000F00700D6E70000C1
:102A200000100140001401402DE9F8439846174674
:102A30000D460446089E24E0701C22D0FDF7BAFF24
:102A4000A0EB0800B0421AD8CEB12068C16849078F
:102A500017D5802D15D0402D13D00168C943090723
:102A60000FD401680025406800902046FFF72EFF34
:102A70000820606484F840500120BDE8F8830320FA
:102A8000FBE72068006835EA000004D00020B84267
:102A9000D2D00020F1E70120F9E7FEE72DE9F04F61
:102AA000ADF22C4D4FF0000ADFF864B10446CDF8CA
:102AB00008A45546D0464FF480174FF0FF39CDF8A3
:102AC00010B4CDF814A400263A460DF20C41684625
:102AD000FFF74BFB98B1012875D0B8F1000F00DD6E
:102AE0006D1C052D71DD1820FFF724FD5FF0180027
:102AF000FFF720FD00200DF22C4DBDE8F08FDDF832
:102B00000C2400254A4507D042B19DF80100F1B2DE
:102B100088420BD0152078E00620E9E70620FFF771
:102B200009FDDDF814040028CDD05AE0BEB12046DE
:102B30000DF10301FDF77FFBDDF80C042146C0F326
:102B40008D020DF58260FDF7B1FCD8B31820FFF7B8
:102B5000F1FC1820FFF7EEFC6FF00100CBE79DF8C9
:102B6000030088B300212B4A0DF1030002E0535407
:102B7000401C491C03780BB1FF29F8DD02F801A0C5
:102B800000210DF58362401C02E05354401C491C97
:102B90000378202B01D01029F7DB02F801A00DF5F6
:102BA00081611046FFF7DFFCDDF808046FF4E821CF
:102BB000C8420BD91820FFF7BDFC1820FFF7BAFC5C
:102BC000484698E710E016E008E01DE05846FDF79B
:102BD0001DFC0620FFF7AEFC432006E00620FFF7B1
:102BE000A9FCDDF8080486E70620FFF7A3FC4FF0F8
:102BF0000108761C68E71820FFF79CFC1820FFF7F7
:102C000099FC6FF0020076E74320FFF793FC5BE747
:102C100000C0000828050020014A024900F023B83E
:102C2000FD2C00081C0000200907090E002804DB09
:102C300000F1E02080F80014704700F00F0000F170
:102C4000E02080F8141D704702E008C8121F08C178
:102C5000002AFAD170477047002001E001C1121F1D
:102C6000002AFBD170472DE9F04116460F46044675
:102C7000002503E03946B047641C6D1C207800280D
:102C8000F8D12846BDE8F08110B50420FEF70DFB11
:102C900006484FF47A710078B1FBF0F004490968F6
:102CA000BDE81040B1FBF0F0FEF70BBB00000020C8
:102CB0000C00002070B5054600244FF47A7603E03E
:102CC000304600F004F8641CAC42F9D370BD70B516
:102CD0004FF0E0240022656964214843A169A3699B
:102CE0008B42FCD002D2A1EB030102E0A5EB03066C
:102CF00031440A4419468242F1D370BD13B54FF6F0
:102D0000FF73012269460248FEF7EAFC00981CBDE9
:102D1000C000002049498AB04FF000600860FDF70C
:102D200057FEFFF781FCFEF7AFFFFEF7C3FFFEF78C
:102D3000E5FFFFF733F8FFF7A7FFFEF743FD082194
:102D40003F48FEF70DFCFEF7E1FD00244FF48C73C5
:102D5000F022214620460094FEF77AFD0A20FFF774
:102D6000A9FF3220FEF7ACFEDFF8D88001214046F3
:102D7000FDF716FE18254FF6FF764FF4FA7748B3A5
:102D80003149D1E90001089106908DF81C408DF879
:102D9000244006A903A8FDF78CFA08A903A8FDF7AB
:102DA0006EFA2AA103A8FDF776FA48B3CDE90045EB
:102DB000334629A28C214A200294FEF717FFCDE961
:102DC0000045334626A2BC2120200294FEF70EFFC8
:102DD00078002FE03846FFF76DFF01214046FDF7F0
:102DE000DFFD00BBCDE90045334621A28C21482000
:102DF0000294FEF7FBFEFDF74FFBFEF7EBFF12E040
:102E00001EA0FFF709FF4FF0E020046144618461D8
:102E100072B621494868214A1060214A1060096849
:102E200081F3088880471FA0FFF7F6FE23A0FFF775
:102E3000F3FE3846FDF744FCF5E7000008ED00E03E
:102E4000780000200000024000800008415050201F
:102E5000464C4147000000004E6F20417070210039
:102E6000506C6561736520446F776E6C6F616400B0
:102E7000426F6F746C6F616400000000415050201D
:102E8000464C4147204F4B2C206A756D7020746F63
:102E9000206170700D0A000000C0000818000020BA
:102EA0001400002072756E20696E20626F6F7420AE
:102EB0007768696C652831290D0A000074686572AD
:102EC00065206973206E6F206C6567616C204150CE
:102ED000500D0A000000000000000000000000008B
:102EE00000000404040404000004000014140A0098
:102EF000000000000000000000000A0A1F0A0A1F6C
:102F00000A0A000000040E1505060C14150E040034
:102F1000000012150D152E2C2A1200000000040AC4
:102F20000A361515291600000202010000000000F3
:102F3000000000001008080404040404080810003D
:102F40000204040808080808040402000000000441
:102F5000150E0E150400000000000008083E0808C9
:102F6000000000000000000000000000020201005C
:102F700000000000003F0000000000000000000012
:102F800000000000000200000020101008080404E7
:102F90000202010000000E1111111111110E0000AA
:102FA0000000040604040404040E000000000E11D6
:102FB00011080402011F000000000E11100C101077
:102FC000110E00000000080C0C0A091F081C00006C
:102FD00000001F01010F1110110E000000000C1263
:102FE000010D1311110E000000001E10080804044A
:102FF0000404000000000E11110E1111110E00004A
:1030000000000E1111191610090600000000000042
:1030100004000000000400000000000000040000A4
:10302000000404000000100804020204081000005C
:10303000000000003F003F0000000000000002040C
:10304000081010080402000000000E11110804040A
:103050000004000000001C22292D2D1D221C000050
:10306000000004040C0A0A1E1233000000000F12B4
:10307000120E1212120F000000001E1101010101B8
:10308000110E000000000F1212121212120F000097
:1030900000001F120A0E0A02121F000000001F1279
:1030A0000A0E0A020207000000001C120101391179
:1030B000120C000000003312121E12121233000014
:1030C00000001F0404040404041F000000003E0864
:1030D0000808080808080907000037120A060A123B
:1030E000123700000000070202020202223F000025
:1030F00000003B1B1B1B15151535000000003B1283
:1031000016161A1A1217000000000E1111111111D3
:10311000110E000000000F12120E02020207000042
:1031200000000E1111111117190E180000000F12D6
:10313000120E0A121237000000001E1101060810BC
:10314000110F000000001F1504040404040E000009
:103150000000331212121212120C0000000033127F
:10316000120A0A0C040400000000151515150E0AB9
:103170000A0A000000001B0A0A04040A0A1B0000D5
:1031800000001B0A0A0A0404040E000000001F09C4
:1031900008040402121F00001C04040404040404B4
:1031A00004041C00000202040404080808101000B3
:1031B0000E0808080808080808080E00040A00009D
:1031C00000000000000000000000000000000000FF
:1031D0000000003F020400000000000000000000AA
:1031E00000000000000C121C123C00000003020250
:1031F000020E1212120E000000000000001C12024B
:10320000120C000000181010101C1212123C0000CA
:1032100000000000000C121E021C00000018240414
:10322000041E0404041E000000000000003C120CF8
:10323000021C221C00030202020E121212370000AE
:103240000004040000060404040E00000008080046
:10325000000C08080808080700030202021A0A0600
:103260000A1300000007040404040404041F0000FF
:1032700000000000000F15151515000000000000EB
:10328000000F12121237000000000000000C121292
:10329000120C000000000000000F1212120E0207B4
:1032A00000000000001C1212121C10380000000068
:1032B000001B06020207000000000000001E020CB6
:1032C000101E000000000004041E0404041C000082
:1032D00000000000001B1212123C00000000000061
:1032E000001B0A0A04040000000000000015150E6F
:1032F0000A0A000000000000001B0A040A1B00006C
:1033000000000000003312120C080403000000004B
:10331000001E0804041E000018080808080C08080D
:103320000808180008080808080808080808080815
:10333000060404040408040404040600160900003A
:10334000000000000000000000000000000000007D
:103350000000000000000000000000080808080845
:10336000080800001818000000486C241200000033
:1033700000000000000000000000002424247F1250
:1033800012127F12121200000000081C2A2A0A0CD6
:103390001828282A2A1C08080000002225151515BF
:1033A0002A585454542200000000000C1212120A31
:1033B00076252911916E0000000606040300000026
:1033C0000000000000000000004020101008080865
:1033D000080808101020400000020408081010100F
:1033E00010101008080402000000000008086B1C00
:1033F0001C6B080800000000000000000808080816
:103400007F0808080800000000000000000000001D
:103410000000000006060403000000000000000099
:10342000FE0000000000000000000000000000009E
:103430000000000006060000000080404020201030
:10344000100808040402020000000018244242424E
:103450004242424224180000000000080E080808FA
:1034600008080808083E00000000003C42424220D4
:1034700020100804427E00000000003C4242201858
:1034800020404042221C000000000020302824245C
:1034900022227E20207800000000007E0202021A14
:1034A00026404042221C0000000000382402021A7C
:1034B00026424242241800000000007E2222101002
:1034C00008080808080800000000003C42424224A6
:1034D00018244242423C00000000001824424242AC
:1034E00064584040241C0000000000000000181830
:1034F0000000000018180000000000000000000894
:10350000000000000008080400000040201008042B
:1035100002040810204000000000000000007F00AE
:1035200000007F00000000000000000204081020DE
:1035300040201008040200000000003C42424640C7
:1035400020101000181800000000001C225A5555C9
:1035500055552D42221C00000000000808181414C4
:10356000243C224242E700000000001F2222221ECB
:1035700022424242221F00000000007C4242010120
:1035800001010142221C00000000001F22424242B1
:1035900042424242221F00000000003F4212121E1F
:1035A00012120242423F00000000003F4212121E6F
:1035B00012120202020700000000003C2222010158
:1035C00001712122221C0000000000E74242424219
:1035D0007E42424242E700000000003E0808080820
:1035E00008080808083E00000000007C10101010B9
:1035F000101010101010110F0000007722120A0E88
:103600000A121222227700000000000702020202C2
:1036100002020202427F0000000000773636363692
:103620002A2A2A2A2A6B0000000000E346464A4A5A
:1036300052525262624700000000001C2241414188
:1036400041414141221C00000000003F42424242F1
:103650003E020202020700000000001C224141411C
:1036600041414D53321C60000000003F4242423E47
:103670001212222242C700000000007C42420204D3
:1036800018204042423E00000000007F4908080820
:1036900008080808081C0000000000E742424242F7
:1036A00042424242423C0000000000E742422224E3
:1036B00024141418080800000000006B4949494907
:1036C0005555362222220000000000E7422424182B
:1036D0001818242442E70000000000772222141466
:1036E00008080808081C00000000007E21201010B7
:1036F00008040442423F000000780808080808084F
:1037000008080808080878000000020204040808F5
:103710000810102020204040001E10101010101023
:103720001010101010101E0000384400000000009F
:103730000000000000000000000000000000000089
:1037400000000000000000FF00060800000000006C
:103750000000000000000000000000000000003C2D
:103760004278444242FC0000000000030202021AB8
:1037700026424242261A00000000000000000038E5
:1037800044020202443800000000006040404078DB
:103790004442424264D80000000000000000003CA7
:1037A000427E0202423C0000000000F08808087ED1
:1037B00008080808083E0000000000000000007C27
:1037C00022221C023C42423C000000030202023A58
:1037D0004642424242E700000000000C0C00000E8E
:1037E00008080808083E00000000003030000038DB
:1037F000202020202020221E00000003020202724E
:10380000120A1612227700000000000E08080808AD
:1038100008080808083E0000000000000000007FC3
:103820009292929292B70000000000000000003BCC
:103830004642424242E70000000000000000003C17
:1038400042424242423C0000000000000000001BD7
:1038500026424242221E02070000000000000078BB
:1038600044424242447840E00000000000000077FB
:103870004C040404041F0000000000000000007C51
:1038800042023C40423E0000000000000008083EAA
:10389000080808080830000000000000000000636D
:1038A0004242424262DC000000000000000000E7EB
:1038B000422424140808000000000000000000EB6F
:1038C0004949555522220000000000000000007602
:1038D00024181818246E000000000000000000E703
:1038E0004224241418080807000000000000007E8D
:1038F00022100808447E000000C020202020201054
:10390000202020202020C0001010101010101010B7
:1039100010101010101010100006080808080810E9
:1039200008080808080806000C32C2000000000061
:103930000000000000000000000000000000000087
:103940000000000000000000000000000000000077
:103950000000000000000000000000000000000067
:103960000000000000000000000000000000000057
:103970006000600060006000600060006000400067
:103980002000200020000000000000006000600017
:1039900060000000000000000000000060066006FB
:1039A000300398018800440000000000000000007F
:1039B0000000000000000000000000000000000007
:1039C00000000000000000000000000000000000F7
:1039D0001002100210021002FE07FE070802080182
:1039E000080108010801FE07FE07040104010401A3
:1039F0000401000000000000000000000000400082
:103A00004000F00158034C03CC034C0058007000F8
:103A1000E000C001C00140034C035C034C034801BB
:103A2000F000400040000000000000000000000026
:103A30000E010A01910091009100510051003A00DD
:103A4000AE03A00250045004480448044804840211
:103A500084030000000000000000000000000000DF
:103A600038006C006C006C006C006C002C00980737
:103A70001C011A01330133016301E300C308C609C5
:103A80003C07000000000000000000000C001C00CB
:103A900010001000080004000000000000000000FA
:103AA0000000000000000000000000000000000016
:103AB0000000000000000000000000000004000200
:103AC0000001800080004000400020002000200015
:103AD00020002000200020004000400080008000E6
:103AE00000010002000400000000000002000400C9
:103AF000080010001000200020004000400040009E
:103B00004000400040004000200020001000100055
:103B10000800040002000000000000000000000097
:103B2000000000004000C0004000460C4E0FD001D5
:103B3000F0015E0F460C4000400040000000000015
:103B40000000000000000000000000000000000075
:103B50000000000000004000400040004000400025
:103B6000FE0F400040004000400040000000000008
:103B70000000000000000000000000000000000045
:103B80000000000000000000000000000000000035
:103B90000000000000000000000000000C001C00FD
:103BA00010001000080004000000000000000000E9
:103BB0000000000000000000000000000000000005
:103BC000FE070000000000000000000000000000F0
:103BD00000000000000000000000000000000000E5
:103BE00000000000000000000000000000000000D5
:103BF0000000000000000000000000001C001C008D
:103C00001C0000000000000000000000000400068E
:103C1000000200030001000180008000400040001D
:103C200060002000200010001000080008000C00B8
:103C30000400060002000000000000000000000078
:103C40000000F00098010C030C03060606060606A9
:103C5000060606060606060606060C030C03980171
:103C6000F000000000000000000000000000000064
:103C7000000040007C0060006000600060006000A8
:103C80006000600060006000600060006000600034
:103C9000FC03000000000000000000000000000025
:103CA0000000F8008401020306030603000300017C
:103CB0008001C0006000200010000802040206021B
:103CC000FE030000000000000000000000000000F3
:103CD00000007800C6008601860180018001C000D6
:103CE0007000800100010003000306030603860143
:103CF000F8000000000000000000000000000000CC
:103D0000000080018001C001A001A0019001880194
:103D1000880184018201FE0F800180018001800101
:103D2000E0070000000000000000000000000000AC
:103D30000000FC0304000400040004000400F4007C
:103D40008C010403000300030603060382018401BF
:103D5000F80000000000000000000000000000006B
:103D60000000E00118030C030C0004000600E6014B
:103D700016030E0606060606060604060C021803BF
:103D8000F000000000000000000000000000000043
:103D90000000F8070C060402040100010001800085
:103DA0008000400040004000600060006000600053
:103DB00060000000000000000000000000000000A3
:103DC0000000F8010C030606060606060C021C039A
:103DD000F000C8010C0306060606060606060C03DC
:103DE000F0010000000000000000000000000000E2
:103DF0000000F0000C010C0306020606060606068B
:103E000006078C0678060006000300030C018C01EF
:103E1000780000000000000000000000000000002A
:103E2000000000000000000000000000E000E000D2
:103E3000E00000000000000000000000E000E000E2
:103E4000E000000000000000000000000000000092
:103E500000000000000000000000000060006000A2
:103E600000000000000000000000000000006000F2
:103E70006000400020002000000000000000000062
:103E80000004000200018000400020001000080033
:103E90000400080010002000400080000001000223
:103EA000000400000000000000000000000000000E
:103EB000000000000000000000000000FE070000FD
:103EC00000000000FE0700000000000000000000ED
:103ED00000000000000000000000000000000000E2
:103EE00004000800100020004000800000010002D3
:103EF00000040002000180004000200010000800C3
:103F000004000000000000000000000000000000AD
:103F10000000E0031806040C040C0C0C0C0C000749
:103F2000800140004000400000000000E000E00090
:103F3000E0000000000000000000000000000000A1
:103F4000E00018030C02CC0564056605A605B6045E
:103F5000B604B604B604B602E4010C040C0218035D
:103F6000F000000000000000000000000000000061
:103F70000000600060005000D000900090008800B9
:103F800088010801F8010403040304020202020686
:103F90000F0F000000000000000000000000000003
:103FA0000000FE008C030C030C030C030C038C01BB
:103FB000FC000C030C020C060C060C060C060C0391
:103FC000FE010000000000000000000000000000F2
:103FD0000000E00318030C060C04040406000600AD
:103FE000060006000600060006040C040C02180376
:103FF000F0000000000000000000000000000000D1
:1040000000007F008C010C030C030C060C060C0650
:104010000C060C060C060C060C060C030C038C019B
:104020007F00000000000000000000000000000011
:104030000000FF030603060406040600860086004F
:10404000FE008600860086000600060406040602BE
:10405000FF0300000000000000000000000000005E
:104060000000FF030603060406040600860086001F
:10407000FE00860086008600060006000600060098
:104080001F00000000000000000000000000000011
:104090000000F00018010C020C02040206000600E9
:1040A00006000600C60F060306030C030C031803E4
:1040B000F000000000000000000000000000000010
:1040C00000000F0F0606060606060606060606068A
:1040D000FE07060606060606060606060606060687
:1040E0000F0F0000000000000000000000000000B2
:1040F0000000FC0360006000600060006000600081
:1041000060006000600060006000600060006000AF
:10411000FC030000000000000000000000000000A0
:104120000000F807C000C000C000C000C000C00010
:10413000C000C000C000C000C000C000C000C0007F
:10414000C000C60066003C00000000000000000047
:104150000000CF038601C600460026001600360088
:104160002E006E004600C60086008601060106038A
:104170008F070000000000000000000000000000A9
:1041800000001F00060006000600060006000600EC
:1041900006000600060006000600060406040602E5
:1041A000FF0300000000000000000000000000000D
:1041B00000000707860386038E038E034E034E031B
:1041C0004A035A035A033A033203320332031203F7
:1041D0008707000000000000000000000000000051
:1041E00000008E0F0C021C021C0234023402640216
:1041F00064024402C40284028403840304030403AB
:104200001F0200000000000000000000000000008D
:104210000000F00098010C030C02060606060606D4
:10422000060606060606060606060C020C0398019C
:10423000F00000000000000000000000000000008E
:104240000000FF000603060606060606060606062A
:104250008603FE00060006000600060006000600B3
:104260001F0000000000000000000000000000002F
:104270000000F00098010C030C0206060606060674
:10428000060606060606060676064C02CC039801CC
:10429000F0008007000300000000000000000000A4
:1042A0000000FF01060306060606060606060603CC
:1042B000FE004600C60086008601060306030606C9
:1042C0000F0E0000000000000000000000000000D1
:1042D0000000F8020C030602060206000E003C0075
:1042E000F800E003800300070206020606060C033E
:1042F000F0010000000000000000000000000000CD
:104300000000FE0762046108610860006000600050
:10431000600060006000600060006000600060009D
:10432000F801000000000000000000000000000094
:1043300000001E070C020C020C020C020C020C0204
:104340000C020C020C020C020C020C020C021801F2
:10435000F00000000000000000000000000000006D
:1043600000000F070602040104010C010C01880083
:104370008800980098005000500070003000200025
:10438000200000000000000000000000000000000D
:104390000000F70E6204420446044604640264020C
:1043A000E402E4029C029C019801980188018800C3
:1043B0008800000000000000000000000000000075
:1043C00000009E070C01080118019000B000600079
:1043D000200060006000D000900088010801040304
:1043E0008E07000000000000000000000000000038
:1043F00000000F0F060404020C0208011801B800A7
:10440000B00070006000600060006000600060004C
:10441000F8010000000000000000000000000000A3
:104420000000FC070C02060302018001800040002E
:104430004000200020001000180008040C040402B2
:10444000FE0300000000000000000000E003200068
:10445000200020002000200020002000200020005C
:10446000200020002000200020002000200020004C
:1044700020002000E0030000000000000000000019
:1044800004000400080008001000100010002000C4
:10449000200040004000C0008000800000010001BA
:1044A0000002000200020004000000007C00400046
:1044B00040004000400040004000400040004000FC
:1044C00040004000400040004000400040004000EC
:1044D000400040007C0000000000600090000801E7
:1044E00000000000000000000000000000000000CC
:1044F00000000000000000000000000000000000BC
:1045000000000000000000000000000000000000AB
:10451000000000000000000000000000000000009B
:10452000000000000000000000000000000000008B
:10453000000000000000FF0F0000000018006000F5
:10454000000000000000000000000000000000006B
:10455000000000000000000000000000000000005B
:10456000000000000000000000000000000000004B
:10457000000000000000000000000000F0010C033B
:104580000C030003E0031C030E03060306038E0B5B
:104590007C0E000000000000000000000000000091
:1045A00008000E000C000C000C000C00CC013C03B9
:1045B0001C060C060C060C060C060C060C021C0352
:1045C000E401000000000000000000000000000006
:1045D000000000000000000000000000F0008C015E
:1045E0008C01860106000600060006020C020C0182
:1045F000F0000000000000000000000000000000CB
:104600000002C003000300030003000378038C03CF
:104610000C030603060306030603060304038C07C4
:104620007801000000000000000000000000000011
:10463000000000000000000000000000E00118037E
:1046400008020C060C06FC070C000C0018041802EB
:10465000E001000000000000000000000000000079
:104660000000C0036006300630003000FE0130005C
:1046700030003000300030003000300030003000BA
:10468000FC0100000000000000000000000000002D
:10469000000000000000000000000000F007D80645
:1046A0008C018C018C019801F8000C00FC00CC03FB
:1046B000060306038E03F80000000000000000005F
:1046C00008000E000C000C000C000C00EC011C0398
:1046D0000C030C030C030C030C030C030C030C0362
:1046E0009E07000000000000000000000000000025
:1046F0000000600060000000000040007C006000DE
:1047000060006000600060006000600060006000A9
:10471000FC0300000000000000000000000000009A
:104720000000C001C001000000000001F001800194
:104730008001800180018001800180018001800171
:1047400080018001CC007C0000000000000000001F
:1047500008000E000C000C000C000C008C038C00F8
:104760008C004C006C005C008C008C010C010C0374
:104770009E07000000000000000000000000000094
:1047800040007C006000600060006000600060002D
:104790006000600060006000600060006000600019
:1047A000FC0300000000000000000000000000000A
:1047B0000000000000000000000000003707EE06C7
:1047C0006606660666066606660666066606660689
:1047D000FF0F0000000000000000000000000000CB
:1047E000000000000000000000000000EE011C03BB
:1047F0000C030C030C030C030C030C030C030C0341
:104800009E07000000000000000000000000000003
:10481000000000000000000000000000F00098010F
:104820000C03060606060606060606060C030C031F
:10483000F000000000000000000000000000000088
:10484000000000000000000000000000EE011C035A
:104850000C060C060C060C060C060C060C031C03BE
:10486000EC010C000C003E00000000000000000005
:1048700000000000000000000000000078028C032F
:104880000C030603060306030603060304038C0356
:10489000780300030003C0070000000000000000D0
:1048A0000000000000000000000000009F03580608
:1048B0003806180018001800180018001800180012
:1048C000FF000000000000000000000000000000E9
:1048D000000000000000000000000000F0031C03C6
:1048E0000C020C023800F000C003040304038C0324
:1048F000FC010000000000000000000000000000BB
:10490000000000002000200030003000FE013000D8
:104910003000300030003000300030003002300213
:10492000E0010000000000000000000000000000A6
:104930000000000000000000000008028E030C03CD
:104940000C030C030C030C030C030C030C039C075B
:1049500078010000000000000000000000000000DE
:104960000000000000000000000000001E070C0214
:104970000801080118019000B000B000600060005C
:104980002000000000000000000000000000000007
:10499000000000000000000000000000F70E6204AC
:1049A000460464026402EC029C019801980198019B
:1049B00008000000000000000000000000000000EF
:1049C000000000000000000000000000BC0718010B
:1049D0001001B00060006000E000900008010803D2
:1049E0009E07000000000000000000000000000022
:1049F0000000000000000000000000009E07080109
:104A00000801080190009000B000600060006000A4
:104A10002000200024001C00000000000000000016
:104A2000000000000000000000000000FC01840104
:104A3000C4004400600020003000180208020C038B
:104A4000FC010000000000000000000000038000E6
:104A50008000800080008000800080008000400096
:104A600020004000800080008000800080008000E6
:104A70008000800000030000400040004000400033
:104A80004000400040004000400040004000400026
:104A90004000400040004000400040004000400016
:104AA0004000400040004000000000000C001000EA
:104AB0001000100010001000100010001000200066
:104AC0004000200010001000100010001000100026
:104AD000100010000C00000000001C002204C204A2
:104AE0008003000000000000000000000000000043
:104AF00000000000000000000000000000000000B6
:104B000000000000000000000000000000000000A5
:104B10000000000000000000000000000000000095
:104B20000000000000000000000000000000000085
:104B30000000000000000000000000000000000075
:104B40000000000000000000000000000000000065
:104B50000000C001C001C001C001C001C001C0010E
:104B600080008000800080008000800080000000C5
:104B70000000000000008001C003C00380010000AD
:104B80000000000000000000000000000000E01C29
:104B9000E01CF01E700E38071803080184000000A6
:104BA0000000000000000000000000000000000005
:104BB00000000000000000000000000000000000F5
:104BC00000000000000000000000000000000000E5
:104BD0000000000020102010201020102010FE7F68
:104BE000FE7F1008100810081008100810081008A0
:104BF000FE7FFE7F0804080408040804080400007F
:104C000000000000000000000000000000000000A4
:104C100000010001C0076019103118311839183926
:104C200038017001E001C0038007000F001D00394A
:104C300000311C311C310C310C11180DE007000142
:104C40000001000100000000000000000000000062
:104C5000000000001C1036186308630C6304630432
:104C6000630263026301361D9C37802280634063C8
:104C7000406320632063306310221836081C000054
:104C80000000000000000000000000000000000024
:104C900000000000F00098018C018C018C018C0157
:104CA0008C00CC007800183E1C08360832086304DB
:104CB0006304C304C303834306438E26781C0000A9
:104CC00000000000000000000000000000001C00C8
:104CD0003C003C003000300010000C0006000000DA
:104CE00000000000000000000000000000000000C4
:104CF00000000000000000000000000000000000B4
:104D00000000000000000000000000000000004063
:104D1000002000100008000C00040006000300033F
:104D200000038001800180018001800180018001F9
:104D3000800100030003000300060006000C0008C9
:104D400000100020004000000000000000000200F1
:104D5000040008001000300020006000C000C00007
:104D6000C0008001800180018001800180018001FC
:104D70008001C000C000C000600060003000100072
:104D80000800040002000000000000000000000015
:104D9000000000000000000000018003800300010B
:104DA0001C713C79783DC0070001C007783D3C7913
:104DB0001C710001800380038001000000000000DE
:104DC00000000000000000000000000000000000E3
:104DD00000000000000000000000000100010001D0
:104DE0000001000100010001FC7F00010001000141
:104DF00000010001000100010000000000000000AF
:104E000000000000000000000000000000000000A2
:104E10000000000000000000000000000000000092
:104E20000000000000000000000000000000000082
:104E300000000000000000001C003C003C003000AE
:104E4000300010000C000600000000000000000010
:104E50000000000000000000000000000000000052
:104E60000000000000000000FE7F000000000000C5
:104E70000000000000000000000000000000000032
:104E80000000000000000000000000000000000022
:104E90000000000000000000000000000000000012
:104EA0000000000000000000000000000000000002
:104EB00000000000000018003C003C00180000004A
:104EC00000000000000000000000000000000040A2
:104ED000006000200030001000180008000C0004E2
:104EE000000600020003000180018000C0004000B5
:104EF0006000200030001000180008000C000400C2
:104F00000600020000000000000000000000000099
:104F100000000000C007600C30181830183018204E
:104F20000C600C600C600C600C600C600C600C6021
:104F30000C601820183018303018600CC0070000C2
:104F40000000000000000000000000000000000061
:104F50000000000000018001F80180018001800153
:104F60008001800180018001800180018001800139
:104F700080018001800180018001C003F81F0000D2
:104F80000000000000000000000000000000000021
:104F900000000000E007101C0818043004300C303A
:104FA0000C300030001800080004000200018000EE
:104FB00040002020102008200430FC1FFC1F0000AF
:104FC00000000000000000000000000000000000E1
:104FD00000000000E003180E0C0C0C180C180C1844
:104FE0000018000C0006C003000E0018001000306E
:104FF00000300C300C300C100C18180CE0030000C2
:1050000000000000000000000000000000000000A0
:1050100000000000000C000E000E000F800E800E3D
:10502000400E600E200E100E100E080E040E040E20
:10503000FE7F000E000E000E000E000E000EC07F60
:105040000000000000000000000000000000000060
:1050500000000000F03FF03F1000100010000800BA
:105060000800C807280C181808100030003000305D
:1050700000300C300C3004180418080CF003000049
:105080000000000000000000000000000000000020
:1050900000000000800FC0102030103018001800F1
:1050A00008000C008C0F6C183C301C600C600C600D
:1050B0000C600C601860182030306018C0070000C9
:1050C00000000000000000000000000000000000E0
:1050D00000000000F83FF83F1C100C08040804040E
:1050E00000040002000200010001000180008000B5
:1050F0008000C000C000C000C000C000C0000000B0
:10510000000000000000000000000000000000009F
:1051100000000000E007300C18180C300C300C3088
:105120001C3038187008E007B007180E0C1C063841
:1051300006300630063006300C18180CE00300006C
:10514000000000000000000000000000000000005F
:1051500000000000E00318040C080C1806100630CC
:1051600006300630063006380C3C1836F031003078
:105170000018001800180C0C0C060C03F0010000BD
:10518000000000000000000000000000000000001F
:10519000000000000000000000000000000000000F
:1051A00000008001C003C003800100000000000077
:1051B0000000000000008001C003C0038001000067
:1051C00000000000000000000000000000000000DF
:1051D00000000000000000000000000000000000CF
:1051E0000000C000C000000000000000000000003F
:1051F00000000000000000000000C000C0008000AF
:10520000800040004000000000000000000000009E
:1052100000000020001000080004000600038001C8
:10522000C0006000300018000C0018003000600062
:10523000C0008001000300060004000800100020E8
:10524000000000000000000000000000000000005E
:10525000000000000000000000000000000000004E
:105260000000FE7F00000000000000000000FE7F44
:10527000000000000000000000000000000000002E
:10528000000000000000000000000000000000001E
:10529000000004000800100020006000C000800131
:1052A00000030006000C001800300018000C000677
:1052B00000038001C000600020001000080004000E
:1052C00000000000000000000000000000000000DE
:1052D0000000C0073018083008600C601C601C60BB
:1052E0001C600030001C000600018000800080006F
:1052F0008000000000008001C003C00380010000A6
:10530000000000000000000000000000000000009D
:1053100000000000C0076018103018200C2F8C4DC2
:10532000864CC64CC64C664C664466446626662669
:105330006615CC1C0C40082018303018C00700003F
:10534000000000000000000000000000000000005D
:1053500000000001C001C001C00140016003200342
:10536000200320033006100610061006F80F080C64
:10537000080C080C0C0C0418041806181F7C0000FC
:10538000000000000000000000000000000000001D
:1053900000000000FE07181C1838183018301830AC
:1053A00018301818180CF80718181830182018603A
:1053B000186018601860186018301818FE0F000088
:1053C00000000000000000000000000000000000DD
:1053D00000000000C0276038103018200C400C403E
:1053E000040006000600060006000600060006008F
:1053F00006000C400C400C2018303018C00700008C
:10540000000000000000000000000000000000009C
:1054100000000000FE03180E18181830183018305D
:1054200018601860186018601860186018601860BC
:1054300018601830183018101818180EFE030000E5
:10544000000000000000000000000000000000005C
:1054500000000000FE3F18301820186018401800A7
:1054600018081808180CF80F180C18081808180055
:10547000180018001840184018201830FE3F00008F
:10548000000000000000000000000000000000001C
:1054900000000000FE7F1870184018C01880180027
:1054A000181018101818F81F1818181018101800CD
:1054B0001800180018001800180018007E000000DE
:1054C00000000000000000000000000000000000DC
:1054D00000000000C013701C101018100C200C20CD
:1054E00004000600060006000600060006FC063062
:1054F00006300C300C30183018303008C00700006F
:10550000000000000000000000000000000000009B
:10551000000000003F7E0C180C180C180C180C181A
:105520000C180C180C180C18FC1F0C180C180C1864
:105530000C180C180C180C180C180C183F7E0000D6
:10554000000000000000000000000000000000005B
:1055500000000000F81F80018001800180018001AF
:105560008001800180018001800180018001800133
:10557000800180018001800180018001F81F00000E
:10558000000000000000000000000000000000001B
:1055900000000000E07F000600060006000600068E
:1055A00000060006000600060006000600060006CB
:1055B00000060006000600060006000600060006BB
:1055C0000E060E038E01FC0000000000000000002B
:1055D000000000007E7C181818081804180618022D
:1055E000180198019801D801B80338031807180664
:1055F000180E180C181C1818183018307EFC0000F3
:10560000000000000000000000000000000000009A
:10561000000000007E001800180018001800180094
:1056200018001800180018001800180018001800BA
:10563000180018001840184018201830FE3F0000CD
:10564000000000000000000000000000000000005A
:10565000000000001FF81C381C381C381C3C343477
:105660003434343434367432643264326432643103
:10567000C431C431C431C430C43084309FFC000014
:10568000000000000000000000000000000000001A
:10569000000000001F7C1C103C10341034107410EB
:1056A0006410E410C410C41184118413041304178B
:1056B0000416041E041C041C041C04181F180000FB
:1056C00000000000000000000000000000000000DA
:1056D00000000000C003300C181808100C300C300B
:1056E000066006600660066006600660066006608A
:1056F00006600C200C3008101818300CC003000095
:105700000000000000000000000000000000000099
:1057100000000000FE0F181818301860186018609C
:105720001860186018301818F80F180018001800C2
:105730001800180018001800180018007E0000005B
:105740000000000000000000000000000000000059
:1057500000000000C003300C18180C100C300C2096
:105760000660066006600660066006600660066009
:105770000660E4612C331C321816300EC007004C52
:10578000007C003800000000000000000000000065
:1057900000000000FE07181C1838183018301830A8
:1057A00018301818180CF80798031803180718066B
:1057B0001806180E180C180C181C18187E78000003
:1057C00000000000000000000000000000000000D9
:1057D00000000000E027303818300C200C200C00AE
:1057E0000C0018007800E003800F001E00380070E5
:1057F000006004600460086018303818C80F0000AA
:105800000000000000000000000000000000000098
:1058100000000000FC3F8C218461824182418001B4
:105820008001800180018001800180018001800170
:10583000800180018001800180018001E00700007B
:105840000000000000000000000000000000000058
:10585000000000003F7C0C100C100C100C100C1001
:105860000C100C100C100C100C100C100C100C1058
:105870000C100C100C100C1008083804E003000089
:105880000000000000000000000000000000000018
:10589000000000003EF818201820182030103010AA
:1058A00030103010600860086008E00CC004C004CC
:1058B000C004800380038003800300010001000016
:1058C00000000000000000000000000000000000D8
:1058D00000000000DFF38661862186218C210C21E7
:1058E0008C238C138C138C134C1358125816580E8F
:1058F000380E380E380E300C10041004100400005E
:105900000000000000000000000000000000000097
:10591000000000007E3E1808380830043004700291
:105920006002E001C001C001800180034003400724
:1059300020062006100C100C081808183E7C0000E9
:105940000000000000000000000000000000000057
:10595000000000007E7C1C10181018083008300C65
:10596000700460046002C002C002C00180018001B6
:10597000800180018001800180018001E00700003A
:105980000000000000000000000000000000000017
:1059900000000000F83F18180818040C040E000658
:1059A0000007000380038001C001C000E000600028
:1059B00070003000382018201C100C18FE1F00004A
:1059C0000000000000000000000000000000C03FD8
:1059D00040004000400040004000400040004000C7
:1059E00040004000400040004000400040004000B7
:1059F00040004000400040004000400040004000A7
:105A00004000C03F00000000000000000000000057
:105A1000000008001800180010003000200060008E
:105A200060004000C0008000800180010001000390
:105A30000002000600060004000C00080018001810
:105A40000010003000200000000000000000FC03F7
:105A50000002000200020002000200020002000236
:105A60000002000200020002000200020002000226
:105A70000002000200020002000200020002000216
:105A80000002FC030000000000000000000080078E
:105A9000C0062008101000000000000000000000F8
:105AA00000000000000000000000000000000000F6
:105AB00000000000000000000000000000000000E6
:105AC00000000000000000000000000000000000D6
:105AD00000000000000000000000000000000000C6
:105AE00000000000000000000000000000000000B6
:105AF00000000000000000000000000000000000A6
:105B0000000000000000FFFF00000000000078001F
:105B1000C0000001000000000000000000000000C4
:105B20000000000000000000000000000000000075
:105B30000000000000000000000000000000000065
:105B40000000000000000000000000000000000055
:105B50000000000000000000000000000000000045
:105B60000000F00318060C0C0C0C000C800F700CDD
:105B70001C0C0C0C060C060C064C0C4FF8380000E4
:105B80000000000000000000000000000000000015
:105B9000000010001E00180018001800180018005F
:105BA0001800180FD818383038601860186018605E
:105BB000186018601860182038307818C80700007E
:105BC00000000000000000000000000000000000D5
:105BD00000000000000000000000000000000000C5
:105BE0000000C007700C181818180C180C000C00D6
:105BF0000C000C000C20182018103008C007000002
:105C00000000000000000000000000000000000094
:105C100000000010001E00180018001800180018DE
:105C20000018E01B301C181818180C180C180C1849
:105C30000C180C180C180818181C307AE009000011
:105C40000000000000000000000000000000000054
:105C50000000000000000000000000000000000044
:105C60000000C007300C181808100C300C30FC3F36
:105C70000C000C000C00182018107018C007000051
:105C80000000000000000000000000000000000014
:105C900000000000003E80C380C0C0C0C000C00043
:105CA000C000FC1FC000C000C000C000C000C00099
:105CB000C000C000C000C000C000C000F80F00005D
:105CC00000000000000000000000000000000000D4
:105CD00000000000000000000000000000000000C4
:105CE0000000C077306C1018181818181818101801
:105CF000300CF00718001800F00FF03F08700C602F
:105D00000C600C603838E00F00000000000000005C
:105D1000000010001E0018001800180018001800DD
:105D20001800980FD818383018301830183018303C
:105D30001830183018301830183018307EFC000039
:105D40000000000000000000000000000000000053
:105D500000000000800380038003000000000000BA
:105D60000001F80180018001800180018001800133
:105D7000800180018001800180018001F81F000006
:105D80000000000000000000000000000000000013
:105D9000000000000038003800380000000000005B
:105DA0000010801F001800180018001800180018B4
:105DB0000018001800180018001800180018001823
:105DC0000018180C1806F003000000000000000086
:105DD000000010001E00180018001800180018001D
:105DE0001800183E180C1806180318019801D8015D
:105DF000380318071806180C181C18187E7C0000A9
:105E00000000000000000000000000000000000092
:105E100000000001F8018001800180018001800103
:105E2000800180018001800180018001800180016A
:105E3000800180018001800180018001F81F000045
:105E40000000000000000000000000000000000052
:105E50000000000000000000000000000000000042
:105E60000800EE1C9C338C318C318C318C318C31A0
:105E70008C318C318C318C318C318C31DE7B00005B
:105E80000000000000000000000000000000000012
:105E90000000000000000000000000000000000002
:105EA00010001E0FD818383018301830183018303D
:105EB0001830183018301830183018307EFC0000B8
:105EC00000000000000000000000000000000000D2
:105ED00000000000000000000000000000000000C2
:105EE0000000C007701C103018300C600C600C6093
:105EF0000C600C600C60183018303018C0070000BF
:105F00000000000000000000000000000000000091
:105F10000000000000000000000000000000000081
:105F200010009E0F5818383018201860186018603C
:105F30001860186018601830383078189807180002
:105F40001800180018007E0000000000000000008B
:105F50000000000000000000000000000000000041
:105F60000000C023303C183818300C300C300C3096
:105F70000C300C300C3008301838303CE033003036
:105F800000300030003000FC000000000000000085
:105F90000000000000000000000000000000000001
:105FA00060007E3C60666061E000E00060006000D0
:105FB000600060006000600060006000FE0700009C
:105FC00000000000000000000000000000000000D1
:105FD00000000000000000000000000000000000C1
:105FE0000000E02730381830182018007000E00357
:105FF000800F001C043004300C301C18EC0F000023
:106000000000000000000000000000000000000090
:106010000000000000000000800080008000C00040
:10602000E000FC1FC000C000C000C000C000C000F5
:10603000C000C000C000C020C0208011000F0000C0
:106040000000000000000000000000000000000050
:106050000000000000000000000000000000000040
:1060600010201E3C183018301830183018301830F6
:106070001830183018301830183830F4E013000099
:106080000000000000000000000000000000000010
:106090000000000000000000000000000000000000
:1060A00000007E3C181818083808300430047002CC
:1060B00060026002E001C001C001C0008000000079
:1060C00000000000000000000000000000000000D0
:1060D00000000000000000000000000000000000C0
:1060E0000000DFF78E630C238C238C239813981306
:1060F00058165816700E700E700E20042004000002
:10610000000000000000000000000000000000008F
:10611000000000000000000000000000000000007F
:106120000000FC3E70087004E004C002C00180035F
:10613000800340076006200C100C18183E7E0000FB
:10614000000000000000000000000000000000004F
:10615000000000000000000000000000000000003F
:1061600000007E7C181818083008300830046004DD
:106170006004C002C002C002800180018001800072
:10618000800080004C003C00000000000000000087
:1061900000000000000000000000000000000000FF
:1061A0000000FC1F0C0C040E040600038003800199
:1061B000C000E0007020302038301C18FC1F0000A8
:1061C000000000000000000000000000000000309F
:1061D000000800040004000400040004000400049B
:1061E0000004000400040002800100020004000416
:1061F000000400040004000400040004000400047F
:10620000000400080030000000010001000100014E
:106210000001000100010001000100010001000176
:106220000001000100010001000100010001000166
:106230000001000100010001000100010001000156
:1062400000010001000100010000000000000C003E
:10625000100020002000200020002000200020004E
:10626000200020002000400080014000200020008D
:10627000200020002000200020002000200020001E
:10628000200010000C00000000003800C400864010
:1062900002610022001C000000000000000000005D
:1062A00000000000000000000000000000000000EE
:1062B00000000000000000000000000000000000DE
:1062C0000000000000000000D6D0200020002000C8
:1062D000FE03220222022202FE03220220002000EC
:1062E0002000BEB0FC010401FC010401FC012000FF
:1062F000FF070401FC01200024013202D4B0FE0794
:106300000204FA0402040204FE05520452044A057F
:1063100086050204FE07B5E710001000FF01110119
:106320001101FF0111011101FF0111041004E00727
:10633000D7D30000FC018000400020002000FF07B0
:1063400020002000200020003800D6D080008000EF
:1063500080008000FC1F841084108410841084103E
:10636000FC1F84108000800080008000BEB0F80F09
:106370000808F80F0808F80F8000FF7F0000F80FEA
:1063800008080808F80F80008410A2204000D4B04C
:106390000000FE3F0220F22702200220FA2F2221D5
:1063A00022212221122912290A2E0220FE3F022038
:1063B000B5E7800080008000FC1F841084108410EA
:1063C000FC1F841084108410FC1F84508040804087
:1063D000007FD7D30000FE1F0008000400028001E8
:1063E0008000FF7F800080008000800080008000AF
:1063F000A0004000D6D000000000000000180000FF
:106400000800000800000800080818F8FF1F180816
:10641000181808181808181808181808181808184C
:10642000F8FF1F0808080008000008000008000026
:106430000800001800001800001800000000BEB09E
:10644000000000000000400006C0FF07400006C03A
:10645000FF07400006C0FF07400802003000FEFFB3
:106460003F000000C0FF07C00002C00002C00002E1
:10647000C0FF0380100080110160100E3010180C56
:106480001E30001C00000000D4B00000000000001E
:10649000080030F8FF1F08001008C010083F10085F
:1064A0000010080010080013C8FF1008221008226E
:1064B00010082210082210082112082114886016E2
:1064C00048C013280010080010F8FF1F0800100033
:1064D0000000B5E700000000000000180000080000
:1064E000000800000800F0FF0F1008041008041056
:1064F0000804100804F0FF0710080410080410082E
:1065000004100804F0FF071008000008100008102D
:1065100000082000183000F01F000000D7D3000052
:1065200000000000000004F0FF0F00000600000162
:1065300000C000002800001800001800001830FEFD
:10654000FF7F001800001800001800001800001855
:1065500000001800001800001800001800001F00BC
:10656000000C00000000D6D0000000000000000079
:106570000080000000800100008001000080010018
:1065800000800100008001001080010CF0FFFF0F6F
:106590003080010430800104308001043080010427
:1065A0003080010430800104308001043080010417
:1065B000F0FFFF07308001043080010400800100FB
:1065C00000800100008001000080010000800100C7
:1065D00000800100008001000080010000800100B7
:1065E0000080000000000000BEB0000000000000BD
:1065F0000000000000000001800100FFFF01000317
:1066000080010003800100FFFF01000380010003FF
:10661000800100FFFF0100818100000003000000F5
:10662000031CFCFFFF3F000040000003C00100FF0F
:10663000FF010003C0000003C0000003C00000FF12
:10664000FF000001410000040100000E710000077E
:106650008101800101076000010E1898011C04E00F
:10666000011800C0000000000000D4B000000000CD
:106670000000000000000008F0FFFF1F3000000CC9
:106680003000000C3000100C30FE3F0C3004000CC9
:106690003000000C3000000C3000000C3000C00C4A
:1066A000F0FFFF0D3030060E3030060C3010060CB7
:1066B0003010060C3010060C3018860C3018860C82
:1066C0003008060D300C860D3006EE0F3002FC0D42
:1066D0003001000CF000000C3000000CF0FFFF0F48
:1066E0003000000C1000000400000000B5E70000BE
:1066F00000000000000000C0000000C0010000C059
:10670000000000C0000000C0000000C00000E0FF6A
:10671000FF0360C0000360C0000360C0000360C0EE
:10672000000360C0000360C00003E0FFFF0360C01F
:10673000000360C0000360C0000360C0000360C0CD
:106740000003E0FFFF0360C0000160C0000000C064
:10675000000800C0001000C0001000C0001800C0F9
:1067600001380080FF1F0000000000000000D7D3A8
:106770000000000000000000000000000000000316
:10678000C0FFFF07000080070000C000000060009D
:106790000000180000000C000080030000800300CF
:1067A00000800100008001080080011CFCFFFF3F09
:1067B00000800100008001000080010000800100D5
:1067C00000800100008001000080010000800100C5
:1067D00000800100008001000080010000800100B5
:1067E00000FC010000E0000000400000000000008C
:1067F0000000000000000000010203040607080971
:1068000000000000010203040A0A0D20415050203C
:10681000466C6167205365742053756363657373B9
:1068200066756C6C79210A0D2D2D2D2D2D2D2D2D9C
:106830002D2D2D2D2D2D2D2D2D2D2D2D2D2D2D2D88
:106840002D2D2D2D2D2D2D2D0D0A00000A0A0D2088
:1068500050726F6772616D6D696E6720436F6D7006
:106860006C65746564205375636365737366756CDA
:106870006C79210A0D2D2D2D2D2D2D2D2D2D2D2D0C
:106880002D2D2D2D2D2D2D2D2D2D2D2D2D2D2D2D38
:106890002D2D2D2D2D0D0A204E616D653A20000005
:1068A0000D0A3D20202020202020202020202020F4
:1068B00020202020202020202020202020202020D8
:1068C00020202020202020202020202020202020C8
:1068D00020202020202020202020202020202020B8
:1068E000202020202020203D000000000D0A3D2017
:1068F0002020202020202020202020202028432964
:1069000020434F50595249474854203230313120AA
:1069100053544D6963726F656C656374726F6E6911
:1069200063732020202020202020202020202020D1
:106930002020203D000000000D0A3D2020202020C6
:106940002020202020202020202020202020202047
:1069500020202020202020202020202020204279BC
:10696000204D4344204170706C69636174696F6E9F
:10697000205465616D202020202020202020203DF3
:10698000000000000D0A3D202053544D33324634A0
:10699000787820496E2D4170706C69636174696FFD
:1069A0006E2050726F6772616D6D696E6720417005
:1069B000706C69636174696F6E202028566572730C
:1069C000696F6E20312E302E3029203D00000000EE
:1069D0000D0A3D3D3D3D3D3D3D3D3D3D3D3D3D3D4A
:1069E0003D3D3D3D3D3D3D3D3D3D3D3D3D3D3D3DD7
:1069F0003D3D3D3D3D3D3D3D3D3D3D3D3D3D3D3DC7
:106A00003D3D3D3D3D3D3D3D3D3D3D3D3D3D3D3DB6
:106A10003D3D3D3D3D3D3D3D000000003C6A0008E0
:106A20000000002020000000482C00085C6A0008DC
:106A300020000020080A0000582C00080100000077
:106A400010000000000000000024F400000000001E
:0C6A50000000000000000000000000003A
:040000050800019955
:00000001FF
